:10063E00202069733A2020200000000000000000F6
:10064E00303030303030303020202020202000005C
:0A065E003031323334353637383985
:03000300013700C2
:1006EB00C200E4F532F522F58CF58AD28CD28E223B
:0D06FB007F507E00EF1F70011EEF4E70F764
:0107080022CE
:0706C1007F381206A67F0539
:1006C800AD071FED600BE4FEEEC3947850F20E8088
:0106D800F72A
:0106D90022FE
:10066800C2B2C2B0C2B1D2B0C2B1D2B28F80C2B22D
:0F067800C2B0C2B1E4F5370537E537B414F92243
:1006A600C2B2C2B0C2B1D2B28F80C2B0C2B1C2B2FF
:0B06B600E4F5370537E537B414F922EE
:0306DA00E493FDA9
:0E06DD00AE05EF2480FF1206A6AF06020668E7
:1004FC00E4FC1206C11206C11206C17F011206C32A
:10050C007F061206A61F1206C87F381206A67F0C9D
:10051C001206A67F401206A6AF04ECFB3395E0FA58
:10052C00743E2BF58274063AF583E493FD1206DDD6
:10053C000CBC10E4E4FCEC2440FFECFB3395E0FA3B
:10054C00744E2BF58274063AF583E493FD1206DDA6
:04055C000CBC10E2E1
:010560002278
:10001E008F0B8E0A8D098C08AD23E4FF1206DDAD21
:10002E00287F491206DDAD297F4A1206DDE47B0AE0
:10003E00FAF9F8AF0BAE0AAD09AC0812026D745E98
:10004E002BF58274063AF5837F471206DAAF0BAEB4
:10005E000AAD09AC08E47B0AFAF9F812026D8F0BAF
:10006E008E0A8D098C08E47B0AFAF9F812026D7477
:10007E005E2BF58274063AF5837F461206DAAF0BD5
:10008E00AE0AAD09AC08E47B0AFAF9F812026D8FDC
:10009E000B8E0A8D098C08E47B0AFAF9F812026DB0
:1000AE00745E2BF58274063AF583E493FD7F451258
:1000BE0006DDAF0BAE0AAD09AC08E47B0AFAF9F81F
:1000CE0012026D8F0B8E0A8D098C08E47B0AFAF9E9
:1000DE00F812026D745E2BF58274063AF583E49382
:1000EE00FD7F441206DDAF0BAE0AAD09AC08E47B12
:1000FE000AFAF9F812026D8F0B8E0A8D098C08E43C
:10010E007B0AFAF9F812026D745E2BF58274063AC8
:10011E00F583E493FD7F431206DDAF0BAE0AAD0906
:10012E00AC08E47B0AFAF9F812026D8F0B8E0A8D79
:10013E00098C08E47B0AFAF9F812026D745E2BF54D
:10014E008274063AF583E493FD7F421206DDAF0B0F
:10015E00AE0AAD09AC08E47B0AFAF9F812026D8F0B
:10016E000B8E0A8D098C08E47B0AFAF9F812026DDF
:10017E00745E2BF58274063AF583E493FD7F41128B
:10018E0006DDAF0BAE0AAD09AC08E47B0AFAF9F84E
:10019E0012026D8F0B8E0A8D098C08E47B0AFAF918
:1001AE00F812026D745E2BF58274063AF583E493B1
:1001BE00FD7F401206DDAF0BAE0AAD09AC08E47B45
:1001CE000AFAF9F812026D8F0B8E0A8D098C087FD0
:0401DE00C80206C885
:1006010020900B752101C294D295D296D297209158
:100611000B752102D294C295D296D29720920B7576
:100621002103D294D295C296D29720930B752104BF
:0D063100D294D295D296C297AF217E0022BE
:10048C003000FDAF22E4FCFDFEFBFA7901F812010D
:10049C00E2A804A905AA06AB07AF8CEFFEE4FCFDAD
:1004AC002BFBEA3EFAED39F9EC38F8AF8AE4FEEBB7
:1004BC002FF536EE3AF535ED39F534EC38F533AB3E
:1004CC0036AA35A934F87F607E370D7C2B12026D6D
:1004DC00EF24F0F531EE34D8F530ED34FFF52FEC98
:1004EC0034FFF52E85313B85303A852F39F538228E
:100561003000FDAF22E4FCFDFEFBFA7901F8120137
:10057100E2A804A905AA06AB07AF8CEFFEE4FCFDD7
:100581002BFBEA3EFAED39F9EC38F8AF8AE4FEEBE1
:100591002FF536EE3AF535ED39F534EC38F533AB68
:1005A10036AA35A934F87F007E3E7D4912026D8F4F
:1005B100278E268D258C248F3B8E3A8D398C3822BF
:10038B003000FDAF22E4FCFDFEFBFA7901F812010F
:10039B00E2A804A905AA06AB07AF8CEFFEE4FCFDAF
:1003AB002BFBEA3EFAED39F9EC38F8AF8AE4FEEBB9
:1003BB002FF536EE3AF535ED39F534EC38F533AF3C
:1003CB0036AE35AD34FC7BA07A867901780012020B
:1003DB006D8F368E358D348C33A804A905AA06ABE8
:1003EB00071201E2A804A905AA06AB07E47F9A7ECF
:1003FB0003FDFC12026D8F2D8E2C8D2B8C2A8F3BC7
:07040B008E3A8D398C382276
:1005C100D2B7C2B77F0A1206C8AFA0E48F0BF50AF3
:1005D100F509F5087F807E967D98FCAB0BAA0AA9E8
:1005E10009A8081201E2E47B33FAF9F812026D8FCF
:0F05F1000B8E0A8D098C088F3B8E3A8D398C3812
:0106000022D7
:10041200758915E4F58CF58A758D3C758BBBD2A96F
:10042200D2ABD2AFD28ED28CF53BF53AF539F53854
:100432001204FC120601E521B4010C752352752841
:100442000A75290A12048CE521B4020C752343753E
:100452002870752946120561E521B4030C75234CF9
:1004620075287575294812038BE521B4040C752390
:100472005175280A75290A1205C1AF3BAE3AAD394A
:0A048200AC3812001E1206EB80A930
:03000B00020007E9
:030007000522329D
:03001B0002068753
:10068700C0E0C0D0758D3C758B830532E532B4145C
:0F06970009C28CC28E753200D200D0D0D0E032B2
:030000000202FFFA
:0C02FF00787FE4F6D8FD75813B020346D1
:1001E200E88FF0A4CC8BF0A42CFCE98EF0A42CFCBC
:1001F2008AF0EDA42CFCEA8EF0A4CDA8F08BF0A43A
:100202002DCC3825F0FDE98FF0A42CCD35F0FCEB98
:100212008EF0A4FEA9F0EB8FF0A4CFC5F02ECD395D
:0F022200FEE43CFCEAA42DCE35F0FDE43CFC22CA
:1002310075F008758200EF2FFFEE33FECD33CDCC84
:1002410033CCC58233C5829BED9AEC99E582984007
:100251000CF582EE9BFEED9AFDEC99FC0FD5F0D6E4
:10026100E4CEFBE4CDFAE4CCF9A88222B800C1B90E
:100271000059BA002DEC8BF084CFCECDFCE5F0CB4C
:10028100F97818EF2FFFEE33FEED33FDEC33FCEB85
:1002910033FB10D703994004EB99FB0FD8E5E4F940
:1002A100FA227818EF2FFFEE33FEED33FDEC33FC2D
:1002B100C933C910D7059BE99A4007EC9BFCE99A21
:1002C100F90FD8E0E4C9FAE4CCFB2275F010EF2F66
:1002D100FFEE33FEED33FDCC33CCC833C810D70766
:1002E1009BEC9AE899400AED9BFDEC9AFCE899F8A1
:0E02F1000FD5F0DAE4CDFBE4CCFAE4C8F92234
:10030B00020412E493A3F8E493A34003F68001F2F2
:10031B0008DFF48029E493A3F85407240CC8C333F3
:10032B00C4540F4420C8834004F456800146F6DFC2
:10033B00E4800B0102040810204080900003E47E4F
:10034B00019360BCA3FF543F30E509541FFEE493B7
:10035B00A360010ECF54C025E060A840B8E493A37E
:10036B00FAE493A3F8E493A3C8C582C8CAC583CAA9
:10037B00F0A3C8C582C8CAC583CADFE9DEE780BE61
:0100060000F9
:00000001FF
